:020000040000FA
:0600000015EF02F01200F2
:02002A000000D4
:04002C00806AF80EE0
:10003000926E0F0EC16E809080948092936AF18EC2
:10004000120093688082809400008084000081BE4A
:10005000FAD7809400008092936A1200D9CFE6FF0D
:10006000E1CFD9FF80928090936AFE0EDB50816EC3
:10007000E8DF8080808400008094070EE66E21EC2B
:1000800002F0E552E552E7CFD9FF1200D9CFE6FFE3
:10009000E1CFD9FF80928090936AFE0EDB50816E93
:1000A000D0DF808400008094070EE66E21EC02F021
:1000B000E552E552E7CFD9FF12003C0EE66EE6DFCF
:1000C000E552080EE66E05EC02F0E5523C0EE66ED7
:1000D000DDDFE552080EE66E05EC02F0E5523C0E5F
:1000E000E66ED4DFE552080EE66E05EC02F0E5524E
:1000F000080EE66ECBDFE552010EE66EC7DFE55275
:10010000060EE66EC3DFE5521200F00E936EF19E0E
:10011000816A020EE66E21EC02F0E55281380F0B87
:1001200000016D6F6C6B6DA104D06D916D436C2BF4
:10013000FAD7040E6C5D23E26CC06EF00F0E936E66
:10014000F19E816A020EE66E21EC02F0E5520F0E7E
:10015000811400016D6F6C6B6DA104D06D916D43C6
:100160006C2BFAD7040E6C5D08E26CC06DF06E511A
:10017000040DF3506D256A6F01D06A6901D06A6978
:10018000F18E1200260EE66EE66A3C0EE66E84ECF8
:1001900001F0E552E552E5521200D9CFE6FFE1CF7A
:1001A000D9FFACA2FED7FE0EDBCFE6FFEEEC01F0EE
:1001B000E552E552E7CFD9FF12000F0EC16E36DFD0
:1001C0007CDF3C0EE66E62DFE5520F0EE66E5EDF10
:1001D000E552826A00016F6BD5DF0001706B6A6BBC
:1001E0000F0E00016A5D37E09EAA08D0B8EC01F05E
:1001F00000016B6F6BC0E6FF31DFE55286DF100E4A
:1002000000016A5D1FE26F511CE1010E6F6F0A0E63
:100210006A5D0CE2300E6A25E66E20DFE552300E94
:1002200000016A25E66EB9DFE5520BD0370E6A256C
:10023000E66E14DFE552370E00016A25E66EADDF8B
:10024000E55203D06F5101E06F6B020EE66ED7EC02
:1002500001F0E552C5D7C00EE66E18DFE552020E7A
:0A026000E66E14DFE552B9D7120074
:06026A002A0EF66E000EE4
:10027000F76E000EF86E00010900F550656F090079
:10028000F550666F03E1656701D03DD00900F55078
:10029000606F0900F550616F0900F550626F090049
:1002A0000900F550E96E0900F550EA6E09000900F1
:1002B0000900F550636F0900F550646F09000900EB
:1002C000F6CF67F0F7CF68F0F8CF69F060C0F6FFBF
:1002D00061C0F7FF62C0F8FF0001635302E164539D
:1002E00007E00900F550EE6E6307F8E26407F9D7FE
:1002F00067C0F6FF68C0F7FF69C0F8FF0001650737
:08030000000E665BBFD712007E
:08030800D9CFE6FFDACFE6FFD2
:10031000E1CFD9FFE2CFDAFFAC6AAB6AFD0EDBB00A
:10032000AC88DBA202D0AC8CAB8CDBB4AC8EDBA691
:1003300002D0AB8801D0AB8ADBA802D0AC8401D05C
:10034000AC949E98DBAC02D09D8A01D09D9A9E9A77
:10035000DBAE02D09D8801D09D98FB0EDB50AF6EC6
:10036000AC8AAB8EE552E5CFDAFFE7CFD9FF1200BA
:10037000D9CFE6FFDACFE6FFE1CFD9FFE2CFDAFF50
:10038000E652F00E00017117ABAC03D07191ABB027
:100390007181ABB47185ABB27187AE50DF6EDF5047
:0E03A000E552E552E5CFDAFFE7CFD9FF1200B4
:0203AE00FF0E40
:1003B000E350036EEF0E01D0F30EE76EE72EDEEF93
:1003C00001F00C0E026EE76AE72EE4EF01F0022E58
:0C03D000E3EF01F0032EDCEF01F012005F
:0403DC00D9CFE6FF90
:1003E000DACFE6FFE1CFD9FFE2CFDAFFACAC04D041
:1003F000AC90000171B3AC80FD0EDB50AD6EE552E8
:0A040000E5CFDAFFE7CFD9FF1200C5
:06040A00FF0EE350036E3B
:10041000480E01D04C0EE76EE72EFED7E76AE72EB6
:0A042000FED7032EF7D700001200EC
:06042A0013EE00F023EECA
:1004300000F0F86A019C35EC01F0DDEC00F0FDD72E
:020440001200A8
:0E044200FF0EE350E84E1200000000D000D084
:0804500000D0E82EFAD71200DB
:020000040030CA
:0E000000100F1F1E008181000FC00FE00F4087
:00000001FF
